:020000040000FA
:100000002E288207003400340034003400341B34BE
:1000100077344034003435346734E03400346A34A3
:10002000CF34C03400349A341D3420340034D534F5
:100030009F34803401341334B234203401344034DA
:100040006F34403401347B34CA3490340134AB34DF
:100050003F3400340134C934C33480348B01073059
:100060009F00C32383168113FF308500860183120E
:10007000AD01AE01AF01B001B101E722E722CB2013
:10008000EB20D201051A4728D2142322D21083165E
:100090009B01AB231A088312BB008316AB231A08FB
:1000A0008312BC008316AB231A088312BD0083168B
:1000B000AB231A088312BE008316AB231A088312DF
:1000C000A0008316AB231A088312A1008316AB236A
:1000D0001A088312A2008316AB231A088312A30006
:1000E00001232F23B022E722E7220508CB000330AB
:1000F0004B05CA00CC01D001A6214B1A8128A120B2
:100100007C28B501B401B30152198B28D21990286B
:100110000130B2009628E830B2000330B3009628D0
:100120000F30B4004230B3004030B200CC189A28EF
:1001300093219C2856216E2101232F23B022E722F0
:100140007C28CC18AD280430D002D7305007031CCF
:10015000AB282830D000B920B4280430D007D730DD
:1001600050070318D001B92001232F23B022E72222
:10017000080050080120A300D00A50080120A20066
:10018000D00A50080120A100D00A50080120A00088
:100190000330D0020800BA23033086000616BA23C3
:1001A0000612033086000616BD23061203308600B1
:1001B0000616BD230612023086000616C02306125C
:1001C00028307C2308307C2301307C2306307C23BC
:1001D0000C307C23080080307C2350308023493051
:1001E000802343308023453080234C308023673088
:1001F0008023653080236E3080238830C3007C23C9
:10020000373080232E308023323080232D308023DE
:1002100033308023303080232030802320308023EF
:10022000C0307C23503080234930802343308023EA
:1002300047308023453080234E3080232030802378
:10024000373080232E3080233230802320308023AB
:1002500020308023203080232030802320308023D2
:1002600020308023AF23C0307C2353308023543090
:10027000802345308023503080233A308023313032
:100280008023483080237A30802320308023203020
:100290008023203080232030802320308023203092
:1002A0008023203080232030802308003208A007DC
:1002B000031C5F29A10F5F29A20F5F29A30A33083E
:1002C000A107031C6629A20F6629A30A3408A20706
:1002D000031C6B29A30A3508A3070800FD30230778
:1002E00003188A2902302302031C92299D30220719
:1002F00003188A2962302202031C9229A5302107A3
:1003000003188A295A302102031C92290030200246
:10031000031C92290030A0005A30A1006230A200D4
:100320000230A3000800B209B309B409B509B20F3D
:100330009E29B30F9E29B40F9E29B50A5621A31FEB
:10034000A529A001A101A201A3010800D21CD4216A
:100350000508CB00C52305084B06031DA62903305D
:100360004B05C9004A060319A6290310CA0D4908FE
:10037000CA064A080239CD004C06CC01CA18C82961
:100380004908CA00CF034F18A629CF18A629D1299A
:100390000230CC004908CA00CF0A4F18A629CF184E
:1003A000A6294908CA0008008519FD29C323851913
:1003B000FD29521DE72952110000D215C6307C23B9
:1003C0004D308023483080237A308023202AD21970
:1003D000F3295215C6307C236B30802348308023AC
:1003E0007A308023202AD211C6307C2348308023E3
:1003F0007A30802320308023202A0519202A1030CB
:10040000D3000519202AB723D30B012A9722CB301A
:100410007C23533080234130802356308023453065
:10042000802344308023AF23CB307C2320308023B3
:1004300020308023203080232030802320308023F0
:10044000851D202A08008030A0009630A100983039
:10045000A2000030A30083169B01AB231A0883126D
:10046000BB008316AB231A088312BC008316AB2390
:100470001A088312BD008316AB231A088312BE002C
:1004800001232F23C430C3007C234330C3008023C7
:100490004130C30080234C30C3008023B022E722C8
:1004A000A621B501B401B3011030B2004B195A2A8C
:1004B0008030B2000000CC18682AB209B309B40930
:1004C000B509B20F682AB30F682AB40F682AB50AB3
:1004D0003208BB07031C712ABC0F712ABD0F712A99
:1004E000BE0A3308BC07031C782ABD0F782ABE0A4F
:1004F0003408BD07031C7D2ABE0A3508BE07051E49
:100500004E2A3B0883169B019A009E2383123C08C7
:1005100083169A009E2383123D0883169A009E2319
:1005200083123E0883169A009E23831208008316C6
:1005300004309B008312200883169A009E238312A6
:10054000210883169A009E238312220883169A009C
:100550009E238312230883169A009E238312080089
:10056000AD01AE01AF01B001B1012030B8003B08D0
:10057000BF003C08C0003D08C1003E08C200031097
:100580003F1CD92A2008AE07031CCB2AAF0FCB2A69
:10059000B00FCB2AB10A2108AF07031CD22AB00F33
:1005A000D22AB10A2208B007031CD72AB10A2308AD
:1005B000B107B10CB00CAF0CAE0CAD0CC20CC10C41
:1005C000C00CBF0CB80BBF2A0030B10008002D30A2
:1005D00084000008BA000830B900BA0C031CF42AE1
:1005E000861506150611F72A861106150611B90B90
:1005F000ED2A840A32300402031CE92A8617861386
:1006000008002030B600A801A901AA01AB01AC0185
:100610000310A00DA10DA20DA30D03182014A80D09
:10062000A90DAA0DAB0DAC0DB603031D182B0800C8
:10063000283084002423840A2423840A2423840A5F
:100640002423840A2423082B03300007B700B7199A
:10065000800030300007B700B71B800008008030F2
:100660007C23203080232B0E0F39303E80232B0833
:100670000F39303E80232C3080232A0E0F39303E34
:1006800080232A080F39303E8023290E0F39303E4F
:1006900080232E30802388307C2329080F39303E78
:1006A0008023280E0F39303E802328080F39303E32
:1006B0008023203080236B308023483080237A30A1
:1006C00080232030802308008601831608308600AE
:1006D000831206138616FF30C50006160608C400EE
:1006E000061200000000061600000612C5030319DA
:1006F0007B2BC4196D2B0800C300D1010613832B7B
:10070000C300511406176423860183160030860047
:1007100083128612061351180617F0308605430E11
:100720000F398604061600000612F03086054308CD
:100730000F39860406160000061208001C158B13DC
:1007400055309D00AA309D009C149C18A52B9C1729
:100750001C119B0A08001C141A089B0A0800B423E9
:10076000B423B423B4230800B723B7230800FF3011
:10077000C500C72B8030C500C72B4030C500C72B34
:100780002030C500C72B1030C5000230C500FF3037
:0C079000C600C60BC92BC50BC72B080008
:02400E00303F41
:10420000CA0017005C00220028000100D600000050
:10421000000000000000000000000000000000009E
:10422000000000000000000000000000000000008E
:10423000000000000000000000000000000000007E
:10424000000000000000000000000000000000006E
:10425000000000000000000000000000000000005E
:10426000000000000000000000000000000000004E
:10427000000000000000000000000000000000003E
:10428000000000000000000000000000000000002E
:10429000000000000000000000000000000000001E
:1042A000000000000000000000000000000000000E
:1042B00000000000000000000000000000000000FE
:1042C00000000000000000000000000000000000EE
:1042D00000000000000000000000000000000000DE
:1042E00000000000000000000000000000000000CE
:00000001FF
